:100000009E01E6287620A0000408A200E1289101C4
:1000100090009F1727308F0010301A2003308F0078
:10002000E8301A208F0164301A208F010A301A201C
:10003000100826288E0011088D0010088C00C5209D
:100040000C08031924289F139F1B0800303E9200C0
:10005000220884000930930003103320920C930B84
:100060002D2803143328841320089F1943280000E7
:10007000031C03011F1920060006200580068417B3
:100080002009800551281F1D030100062005800658
:1000900084172008031C03010006200580061F1793
:1000A0001F1F1F131F0D06398C005F208D008C0A47
:1000B0005F201F1F97288C000230AA20972800304D
:1000C0008A000C088207013471340334113400347F
:1000D00038340C34D5347620800472287620FF3AE8
:1000E00080057328FF3A84178005E12894000630C4
:1000F00094190530840000308A00140807398207FB
:100100000134023404340834103420344034803450
:100110008F018E006400FF308E07031C8F07031CC5
:10012000080003308D00DC3097208A288D01E83EDE
:100130008C008D09031CA128FC308C0703189D2816
:100140008C078D0F9C288C18A5288C18A7280C18B4
:10015000A928080003108D0C8C0CFF3E031DAA2853
:100160000C08E1288D018F018E00BA200239031D91
:10017000FF30E1280F080D02031DC2280E080C02F3
:1001800003190234031C043401341030920091012D
:1001900090010D0D900D910D0E0890020F08031C9B
:1001A0000F0F91020318DB280E0890070F080318A1
:1001B0000F0F910703108C0D8D0D920BC9280C08A1
:1001C000E1288313031383126400080001306E20BA
:1001D00003308F00E83089200030022006309F0075
:1001E000FE3027200130272003308F00E83089209F
:1001F0000030022006309F00FE302720803027206C
:100200003130272030302720203027204D30272044
:10021000693027206E3027202030272049302720C2
:1002200044302720203027205430272069302720D1
:100230006D302720653027207230272000300220C3
:1002400006309F00FE302720C03027204230272074
:10025000793027203A302720203027205730272098
:1002600044302720343027204230272049302720AF
:1002700053302720203027202030272007308F00C0
:10028000D03089200030022006309F00FE30272029
:10029000013027200030022006309F00FE3027204A
:1002A00080302720493027206430272065302720E0
:1002B0006E302720743027206930272066302720B1
:1002C0007930272020302720493027206E30272002
:1002D0005830A4000230A5000030022006309F00F4
:1002E000FE302720C0302720250891002408082050
:1002F00020302720533027206530272063302720E7
:100300006F3027206E30272064302720733027205D
:100310002030272003308F00E83089200130A402EC
:100320000030031C013EA50224088C0025088D0026
:1003300001308F00E030B420031DE22924088C0036
:1003400025088D0001308F006830B420031DE52999
:1003500024088C0025088D008F01F030B420031D87
:10036000E82924088C0025088D008F017830B420FE
:10037000031DEB2924088C0025088D008F01003017
:10038000B420031DEE290030022006309F00FE300D
:100390002720C0302720250891002408082020307D
:1003A00027205330272065302720633027206F30E7
:1003B00027206E30272064302720733027202030FC
:1003C00027206C2904306B206C2905306B206C29A8
:1003D00006306B206C2907306B206C29003002201E
:1003E00006309F00FE3027200130272000300220F9
:1003F00006309F00FE3027208030272054302720F1
:10040000693027206D3027206530272020302720B5
:10041000543027206F3027202030272049302720D4
:1004200064302720653027206E3027207430272045
:1004300069302720663027207930272000300220BD
:1004400006309F00FE302720C03027205030272064
:100450007230272065302720733027207330272003
:100460002030272052302720653027207330272066
:10047000653027207430272008306B2001306B2036
:1004800007308F00D030892001306E2000300220EC
:1004900006309F00FE302720013027200030022048
:1004A00006309F00FE302720803027204130272053
:1004B0006D302720613027207430272065302720B9
:1004C00075302720723027202030272052302720F7
:1004D0006130272064302720693027206F302720A3
:1004E000203027200030022006309F00FE302720D9
:1004F000C030272053302720743027206130272038
:1005000074302720693027206F3027206E30272055
:100510002030272057302720443027203430272010
:1005200042302720493027205330272007308F00C2
:10053000D03089200030022006309F00FE30272076
:10054000013027200030022006309F00FE30272097
:100550008030272054302720693027206D30272015
:100560006530272020302720543027206F30272067
:10057000203027204930272064302720653027206D
:100580006E302720743027206930272066302720DE
:10059000793027200030022006309F00FE302720CF
:1005A000C030272050302720723027206530272088
:1005B0007330272073302720203027205230272007
:1005C000653027207330272065302720743027209E
:0E05D00007308F00D0308920462A6400ED2AC3
:084000007F007F007F007F00BC
:04400E00F53F010079
:00000001FF
